:107800000C942A3C0C94453C0C94453C0C94453C0F
:107810000C94453C0C94453C0C94453C0C94453CE4
:107820000C94453C0C94453C0C94453C0C94453CD4
:107830000C94453C0C94453C0C94453C0C94453CC4
:107840000C94453C0C94453C0C94453C0C94453CB4
:107850000C94453C11241FBECFE5D8E0DEBFCDBF60
:1078600010E0A0E6B0E0E2EDFDE702C005900D9269
:10787000A036B107D9F710E0A0E6B0E001C01D9234
:10788000A036B107E1F70C94303D0C94003CAF9268
:10789000BF92CF92DF92EF92FF920F931F93CF93FD
:1078A000DF93CDB7DEB7C058D0400FB6F894DEBF37
:1078B0000FBECDBF5C016A016534E9F5EE24FF24FB
:1078C000EA14FB0468F48E010F5F1F4F0E0D1F1D9D
:1078D0000E94E33ED8018C930894E11CF11CF0CF88
:1078E00087B799279C012170307080FDF9CF79010D
:1078F0002A153B0508F05DC0FE013196D6018C913A
:107900008EBB8D919C91892F99278FBB80818DBBD8
:10791000E29AE19AE199FECFD6018D919C9111975F
:1079200001968D939C930894E11CF11C3196EA1406
:10793000FB0420F33EC0663409F03EC0FA01E0804B
:10794000F180EE0CFF1CF182E0820E94E33E082FE2
:1079500011270E94E33E9927982F8827082B192B7F
:1079600021E0D6018D919C910801FC0120935700E4
:10797000E89511240296F601918380838EEF9FEFA4
:10798000A80EB91EA114B10401F785E0F701809398
:107990005700E89507B600FCFDCF81E180935700C2
:1079A000E895D6018D919C911197969587958D9329
:1079B0009C938DE090E002C08FE390E0C058DF4FD1
:1079C0000FB6F894DEBF0FBECDBFDF91CF911F91F0
:1079D0000F91FF90EF90DF90CF90BF90AF90089500
:1079E0000F931F93CF93DF938C01EA016534A1F4C9
:1079F00088818EBB88819981892F99278FBB888147
:107A00009981019699838883E09A8DB30E94DE3E26
:107A10000150104069F71FC06634E9F488819981EC
:107A2000880F991F99838883E881F98184910E9446
:107A3000DE3EE881F981319684910E94DE3E8881A4
:107A400099810296998388830250104069F7969530
:107A5000879599838883DF91CF911F910F91089526
:107A6000CDE5D8E0DEBFCDBFCC24DD248FEF8BBBCE
:107A700080E38ABB8CE988BB8BE587BB83EC85BB45
:107A800080EC84BB8FE282BB82EF81BBDE9A0E94D6
:107A9000D93EAE98CE9982C10E94E33E813611F460
:107AA00089E579C1813469F40E94E33E9927182F52
:107AB00000270E94E33E9927082B192B1A8309837C
:107AC00069C08536A1F41A82198223E007B600FC4A
:107AD000FDCF89819A81FC0120935700E895805859
:107AE0009F4F9A8389838050984780F353C0823692
:107AF00041F489E50E94DE3E80E00E94DE3E80E89F
:107B00004AC18234A1F40E94E33E9927F82EEE2464
:107B10000E94E33E9927E82AF92A0E94E33E682F53
:107B2000AE014F5F5F4FC7010E94473C34C18736AB
:107B3000A1F40E94E33E9927F82EEE240E94E33E32
:107B40009927E82AF92A0E94E33E682FAE014F5F89
:107B50005F4FC7010E94F03C9FCF8235A9F407B662
:107B600000FCFDCF81E180935700E895E981FA811F
:107B7000EE0FFF1F319684910E94DE3EE981FA816B
:107B8000EE0FFF1F849164C0833631F40E94E33E00
:107B9000E82EFF248DE0FFC08334F9F40E94E33E19
:107BA0009927982F8827E82AF92A07B600FCFDCFE5
:107BB00041E029813A81C901042E02C0880F991F32
:107BC0000A94E2F70701FC0140935700E89511245D
:107BD0002F5F3F4F3A832983DDCF8D36A9F429816A
:107BE0003A818CE32030380720F08FE30E94DE3E9C
:107BF000D1CF07B600FCFDCF85E0220F331FF9017E
:107C000080935700E895C6CF8434B9F407B600FCDA
:107C1000FDCF89818EBB89819A81892F99278FBB5E
:107C20000E94E33E8DBBE29AE19AE199FECF898101
:107C30009A8101969A838983ADCF843689F48981AC
:107C40008EBB89819A81892F99278FBBE09A8DB34A
:107C50000E94DE3E89819A8101969A8389831CCF96
:107C60008C3669F407B600FCFDCF0E94E33E99E034
:107C7000E1E0F0E0082E90935700E8958BCF823733
:107C800051F407B600FCFDCF89E0E1E0F0E080931D
:107C90005700849180C0863451F407B600FCFDCFB4
:107CA00089E0E0E0F0E080935700849174C08E3466
:107CB00051F407B600FCFDCF89E0E3E0F0E08093EB
:107CC0005700849168C0813551F407B600FCFDCFA0
:107CD00089E0E2E0F0E08093570084915CC0803559
:107CE00009F458CF8C3409F455CF853469F407B6BC
:107CF00000FCFDCF81E180935700E8958DE00E9464
:107D0000DE3EF6010995C8CE803711F483E543C005
:107D1000843729F48FE70E94DE3E80E03CC088373C
:107D200021F40E94E33EDD9835CF893721F40E948B
:107D3000E33EDD9A2FCF843519F40E94E33E2ACF2B
:107D40008335A1F481E40E94DE3E86E50E94DE3E9A
:107D500082E50E94DE3E82E40E94DE3E8FE40E94C5
:107D6000DE3E8FE40E94DE3E84E515C0863529F4B0
:107D700081E30E94DE3E85E30EC0833741F482E05A
:107D80000E94DE3E85E90E94DE3E8EE104C08B311A
:107D900009F482CE8FE30E94DE3E7ECE07B600FC61
:107DA000FDCF81E180935700E895F60109950C9489
:107DB000E83E83E389B988E18AB908958CB95E9B6E
:107DC000FECF5E9A08955F9BFECF8CB199270895F0
:027DD000FFCFE3
:040000030000780081
:00000001FF
